:020000040000FA
:020000000528D1
:08000800B02A831203138501E5
:1000100086018701880189019F01831606309F00B0
:100020003F3085008601F03087003F30880089012D
:100030008730810083128B128B172630AE00A80107
:100040004F20B301B20109142808031D30282621CE
:10005000851E5B20051EBF20071F0621871F162156
:10006000071EDC20871EF120851DCD201030A30047
:10007000C3014430430784000008FF3A8600430868
:1000800087009422FF308600C30AA30B3928A81CDE
:10009000242839210914A6220910A8102428103078
:1000A000A300C10144304107840000308000C10A30
:1000B000A30B522808002D08031D60281030AD0046
:1000C000AD0BB728B101B001A7015208031D6F287D
:1000D00053080319A428D200D30127147228530807
:1000E000031D7D283108002452020319B128B10AEA
:1000F0003108363C03187228A428B00A0310310DC9
:100100003C245202031D8B280310310D013E3C2478
:1001100053020319B128B10A31084F3C03187E2855
:10012000B101B00A0310310D00255202031D9F28B2
:100130000310310D013E002553020319B128B10A05
:100140003108233C031892280A30A400B820A822C2
:10015000A40BA62827080319B7285208D300D201F8
:10016000B7283108B3003008B200C221B820080017
:100170000910A822091424080319AA2208002D082E
:10018000031DC4281030AD00AD0BCC282E08AF00E5
:1001900081018B160910AA2208002D08031DD22800
:1001A0001030AD00AD0BDB288B12280803194F204F
:1001B0000914A801AA2208002D08031DE128103007
:1001C000AD00AD0BF02828080319ED2898302E0259
:1001D0000319F0280310AE0DEF28B3037D21B820DA
:1001E00008002D08031DF6281030AD00AD0B0529C1
:1001F00028080319022913302E02031905290310B8
:10020000AE0C0429B30A3921B82008002D08031DBB
:100210000B291030AD00AD0B15293208023C03301C
:10022000031D0530B3027D21B82008002D08031DF1
:100230001B291030AD00AD0B25293208023C0330DC
:10024000031D0530B3073921B8200800BF30332122
:1002500003192C29D20631297F3033210319322981
:10026000D306B8200800880094220808FF3A3F39D6
:1002700008003208031D4D293308363C0318432972
:10028000B20AB301572933080024FF39031D4A2954
:10029000B30A3C29D200D3017B29013C031D662906
:1002A00033084F3C03185729B20AB3016D290310D4
:1002B000330D3C24FF39031D5F29B30A5029D200B6
:1002C0000310330D013E3C24D3007B293308233C2B
:1002D00003186D29B201B30143290310330D002522
:1002E000FF39031D7529B30A6629D2000310330DA7
:1002F000013E0025D300C22108003208031D9229C7
:10030000330D031C88290230B2002330B300B22918
:1003100033080024FF39031D8F29B3038829D20035
:10032000D301C029013C031DAB29330D031C9C29BB
:10033000B2033630B30088290310330D3C24FF3953
:10034000031DA429B3039C29D2000310330D013EE1
:100350003C24D300C029330D031CB229B2034F3013
:10036000B3009C290310330D0025FF39031DBA2962
:10037000B303B229D2000310330D013E0025D30090
:10038000C22108003208031DD6290630B40000300F
:10039000B5007D228C22B6000630B4000130B500D5
:1003A0007D228C22B7002C2271222B2A013C031DB6
:1003B0000D2A3308223C031CEE290630B4006E30AF
:1003C000B5007D228C22B6000630B4006F30B50037
:1003D0007D228C22B7002C2271222B2A0630B400F9
:1003E000B430B50080228C22B6000630B400B5309F
:1003F000B50080228C22B7002C220630B400B63023
:10040000B50080228C22B6000630B400B730B500AB
:1004100080228C22B7002E222B2A0730B4006830AD
:10042000B50083228C22B6000730B4006930B500D5
:1004300083228C22B7002C220730B4006A30B5002A
:1004400083228C22B6000730B4006B30B5008322C3
:100450008C22B7002E22080001302F2A0230A9007A
:100460000830A400B80139303807840090228A117E
:100470008000B80AB70A0319B60AA40B332A8030E1
:10048000AC000830A400290B482A6D2244304A2AC7
:1004900071224C30C100C2003930B80038088400E5
:1004A0000008AB000830A500290303195A2A0630BA
:1004B000A500AB0DAB0D031C622A410884000008A7
:1004C0002C048000C10AA50B5A2A0310AC0CB80AF0
:1004D0004208C100A40B4E2A08000830A600443090
:1004E000742A0630A6004C30C10041088400003058
:1004F0008000C10AA60B752A08000310330D882A54
:1005000023303302842A3308B1000310B10D310DBA
:10051000B5070318B40A080034088A0035088200B9
:1005200036088A00370882000130A00000006430DD
:100530009C2A0230A000F930A10000000000A10BAD
:100540009D2AA00B9B2A08000530AB2A0A30AB2A53
:100550003230AB2AC830A2009922A20BAC2A080084
:10056000F0000308F100831203130B1D05280B1183
:100570008101AF0BC02A2E08AF00B30A2814A814BB
:0A05800071088300F00E700E0900F0
:10080000AA0004308A002A088207203430342434B5
:10081000343414342134313425343534153423340C
:1008200033342734373417342A343A342E343E34B0
:100830001E34283438342C343C341C3429343934B4
:100840002D343D341D342B343B342F343F341F348E
:100850000C3400340D3400340E3422343234263457
:10086000363416340834183400341A340A340B344D
:100870001034123403341334AA0004308A002A08D6
:1008800082070234213402343134023425340234F4
:100890003534023415340234233402343334023410
:1008A0002734023437340234173402342A34023401
:1008B0003A3402342E3402343E3402341E340234CC
:1008C00029340234393402342D3402343D340234B4
:1008D0001D34013429340134393401342D340134C8
:1008E0003D3401341D340F3420340F3430340F3490
:1008F00024340F3426340F3422340F3434340F347C
:1009000036340F3432340F3414340F341634113477
:100910002034113430340034003411343434113480
:10092000143411342134113431340034003411348E
:1009300035341134153411342A3411343A34113425
:100940002E3411343E3411341E3411342934113410
:10095000393405340D3411343D3411341D3413341D
:1009600029341334393407340D3413343D341334FB
:100970001D34003400340034003413342E34043475
:10098000343400340034133421340034003405345A
:100990002E3404343734003400340034003404344A
:1009A0003A3407342E3404343E34003400340034F6
:1009B000003406343A3402342434063437340034F4
:0209C000003401
:100A0000AA0005308A002A088207043421340434FD
:100A100025340434153404342334043427340434A2
:100A2000173404342A3404342E3404341E34043489
:100A3000283404342C3404341C340434293404346D
:100A40002D3404341D3404342B3404342F34043452
:100A50001F34043422340434263404341634063467
:100A60002134063425340634153406342334063450
:100A700027340634173406342A3406342E34063428
:100A80001E340634293406342D3406341D3405341E
:0A0A9000293405342D3405341D34DB
:100C000008340034083408340834103408341834F4
:100C10000834203408342834083430340834383464
:100C200008344034083448340834503408345834D4
:100C30000834603408346834083470340834783444
:100C400008348034083488340834903408349834B4
:100C50000834A0340834A8340834B0340834B83424
:100C60000834C0340834C8340834D0340834D83494
:100C70000834E0340834E8340834F0340834F83404
:100C80000934003409340834093410340934183470
:100C9000003400340934203400340034093428345A
:100CA0000934303409343834093440340934483490
:100CB0000934503409345834093460340034003471
:100CC0000934683409347034093478340A34F83417
:100CD0000A3450340A3458340A34603409348034C5
:100CE0000934883409349034093498340934A034F0
:100CF0000934A8340934B0340934B8340934C03460
:100D00000934C8340934D0340934D8340934E034CF
:100D10000934E8340934F0340934F8340A3400343E
:100D20000A3408340A3410340A3418340A342034AB
:100D30000A3428340A3430340A3438340A3440341B
:100D40000A3468340A3470340A3478340A3480340B
:100D50000A3488340A3490340A3498340A34A0347B
:100D60000A34A8340A34B034083410340A34B8349D
:100D7000083410340A34C0340034003400340034F1
:100D8000083410340A34D034083410340A34D834D7
:100D9000083438340A34B834083438340A34C034A7
:100DA0000034003400340034083438340A34D03489
:100DB000083438340A34D834083488340A34B8341F
:100DC000083488340A34C034083498340A34C834B7
:100DD000083488340A34D034083488340A34D83497
:100DE0000834D8340A34B8340834D8340A34C03417
:100DF0000834D8340A34E8340834D8340A34D034C7
:100E00000834D8340A34D8340A3448340A34B8346C
:100E10000A3448340A34C0340A3448340A34E834D2
:100E20000A3448340A34D0340A3448340A34D834C2
:100E30000034003400340034003400340034003412
:100E40000934F0340A34C834083408340A34D0344D
:100E50000034003400340034093490340A34B83497
:100E60000034003400340034083490340A34E83458
:100E7000083458340A34D034003400340034003498
:100E80000034003400340034083490340A34C03460
:100E90000934E8340A34E834083480340A34D0346D
:100EA00000340034003400340034003400340034A2
:100EB0000934E8340A34C0340A3448340B3400347A
:100EC0000934B0340A34D0340034003400340034EF
:100ED000083430340A34E034083430340A34E83426
:100EE000083430340A34F034083458340A34E034E6
:100EF000083458340A34E834083458340A34F034A6
:100F0000083480340A34E034083480340A34E83455
:100F1000083480340A34F0340834A8340A34E03415
:100F20000834A8340A34E8340834A8340A34F034D5
:100F30000834D0340A34E0340834D0340A34E83485
:100F40000834D0340A34F0340834F8340A34E03445
:100F50000834F8340A34E8340834F8340A34F03405
:100F6000093438340A34E034093438340A34E83483
:100F7000093438340A34F034093488340A34E0341B
:100F8000093488340A34E834093488340A34F034B3
:100F90000934B0340A34E0340934B0340A34E83463
:100FA0000934B0340A34F0340934D8340A34E03423
:100FB0000934D8340A34E8340934D8340A34F034E3
:100FC0000A3400340A34E0340A3400340A34E83491
:100FD0000A3400340A34F0340A3428340A34E03451
:100FE0000A3428340A34E8340A3428340A34F03411
:1010000010347E34103412343E3455345934323472
:10101000403444344234423441344134493430342D
:101020003C3400347C340234023402340434183446
:10103000383400347E3404340834183428344734C7
:101040002034FA3421343C346234A134A13466347F
:1010500020342034FA3425342534243424344834DC
:1010600010347E3408347E3404343C3440343E340E
:101070000434083410342034203410340834043458
:10108000043484349F348434843484348434483441
:1010900000343C34023400340034403440343E34B4
:1010A00010347E34083404343E34403440343E340A
:1010B00020342034203420342034203422341C3492
:1010C0000834FE3408343834483438340834303482
:1010D00004342434FF3424342434203420341E34A3
:1010E0003C34083410347E340834103410340C345A
:1010F00020347C342034273420344034483447347E
:101100002034FC34203420343C34023402343C3467
:1011100000341E34E1340134013401341E3400340F
:101120000034FE34083410341034103408340634DB
:1011300020342034163418342034403440343E34C3
:101140002034F0344234493488343C344A3438341E
:1011500040345E3441344034403450344F342034D1
:10116000083448347C344A34AA349634AB3444349A
:1011700020342034EC34323422346634AA3425341A
:1011800000341C342A344934493449344934323423
:10119000043484349F34843484349E34A5345C34E1
:1011A0000034E03426342534443444344434383470
:1011B000003410340834103410344A344934913433
:1011C0000034003430344834843403340034003480
:1011D00000349F3484349F3484349E34A5345C348A
:1011E00008347E3408347E3408343C344A3438348D
:1011F00000347034123412347E34933492346434B4
:101200002034FA3421346034A034623422341C3463
:10121000003448347E344934A9349134B1344634EE
:1012200010347E3410347E341034103412340C34C4
:1012300000342834FE34293421342234103410345C
:1012400008340834BE34C934893489344A341034FB
:10125000083408340E34083408343C344A3430340A
:1012600008342434203420343C34023402343C34F6
:101270000434223422342234223402340434183424
:101280003E34043408343C3402341A3426341C34DA
:1012900020342834F434243424346434A5342234FF
:1012A0003E34043408343C340234023422341C34D6
:1012B00020342034EE34313421346134A1342634E6
:1012C0003C3408343C3452349134A7344934063425
:1012D0003C3408343C3402343C3420346C34933491
:1012E00020347C34203436344834183420341E34CE
:1012F00008341034103420343034493449344634FE
:1013000023342034FA342534253424342434483426
:1013100013347E3408347E3404343C3440343E3458
:1013200004340B34103420342034103408340434A2
:10133000073484349F34843484348434843448348B
:1013400003343C34023400340034403440343E34FE
:1013500013347E34083404343E34403440343E3454
:1013600026342034203420342034203422341C34D9
:101370000B34FE34083438344834383408343034CC
:1013800007342434FF3424342434203420341E34ED
:101390003C340B3410347E340834103410340C34A4
:1013A00023347C34203427342034403448344734C8
:1013B0002334FC34203420343C34023402343C34B2
:1013C00003341E34E1340134013401341E3400345A
:1013D0000034FE3408341334103410340834063426
:1013E00023342034163418342034403440343E340E
:1013F000033484349F34843484349E34A5345C3480
:101400000334E0342634253444344434443438340A
:10141000033410340834103410344A3449349134CD
:10142000033400343034483484340334003400341A
:1014300003349E3484349F3484349E34A5345C3425
:10144000023485349E34843484349E34A5345C3430
:101450000234E534223426344534443444343834B8
:10146000023415340A34103410344A344934913477
:1014700002340534323448348434033400340034C4
:1014800002349D3486349F3484349E34A5345C34D5
:1014900013341034FE348234823402340434183469
:1014A0000034003400340034FE340034003400349E
:1014B000003400340034003440342034103410340C
:1014C000003400340034003430344834483430348C
:1014D00008341834083408340834083408341C3408
:1014E0003C34423402340C341034203440347E34E2
:1014F0003C34423402343C340234023442343C340E
:1015000004340C341434243444347E340434043429
:101510007E34403440347C340234023442343C342F
:101520003C34423440347C344234423442343C34DF
:101530007E34023404340834083410341034103447
:101540003C34423442343C344234423442343C34FD
:101550003C34423442343E340234023442343C346B
:101560003C344234423442344234423442343C34D7
:10157000003410347C3412343C345A343234003465
:1015800000340034003444344234423420340034D3
:1015900000341C3400343C34023402341C34003433
:1015A0000034183400343C34083418342634003401
:1015B000003414347A3410343C34523474340034EB
:1015C000003428347C342A34223414341034003467
:1015D000003410345C347234523414342034003407
:1015E000003408340E3408343C344A34383400347F
:1015F0000034003400341C34623402341C340034AF
:10160000003400340034003400340034003400343A
:02400E00323F3F
:00000001FF
